:020000040000FA
:040000004DEF01F0CF
:0800080067D1046E7F0B04BCFC
:100010008008280FF66EF76A000EF722F86A0800CB
:10002000F55004BE00081200000306090C10131658
:10003000191C1F2225282B2E313336393C3F4144D1
:1000400047494C4E515355585A5C5E60626466682D
:100050006A6B6D6F70717374757678797A7A7B7C60
:100060007D7D7E7E7E7F7F7F7F00086E0950085EEB
:10007000D8A009061250115ED8A01206D8900932F5
:100080000832D890123211320150066E0250076EBB
:100090000C6A0D6A0E6A0F6A106A0B6A0F0EEA6E1E
:1000A0000050120FE96E031CEF16100E0000E82E30
:1000B000FED700D0000008500D2609500E22115026
:1000C0000F26125010220E50A0DF800F056E105028
:1000D0009CDF800F0524E8300B2600C0E9FFEF50BD
:1000E0000310D8A00318EF6E0C04D8A0D20E0C6E2B
:1000F000E86A065A075AD9E21200E836E8363C0B9D
:100100000109C212C009C216C050F80B0309C06E23
:10011000320E15D8C282C2B2FED7C4CF12F0C3507D
:10012000116E1200076A066EFF0E0626072200D027
:10013000D8A01200030E056EE60E02D8F5D7056AA8
:10014000FE0F046E000000D000D0E86A055AD8A067
:100150001200040600D000D0F5D7E988E92AEC1691
:1001600012001750156E1B18216E1650D8A41A5085
:100170003CE016267E0E03E3165E03E338D0165EDF
:1001800033E319C013F018C014F0158E1B8E196AD2
:10019000186A176A180E206E15321432133206E3ED
:1001A0001D5019261C5018221B50172217321832C6
:1001B0001932202EF1D717BE07D019361836173648
:1001C000165212E0160615341FAC17D016E3193E6E
:1001D00014D0183E12D0173E10D0D88017321832E3
:1001E0001932163E0AD003D01F84166A02D01F822D
:1001F0001668196A186A800E176E21AE179E19507C
:100200001200186A196A960E206E219E19AE07D048
:10021000D880000E1656175618561956218E1952A8
:1002200018E01FAC0DD019AE0BD0172A09E1182A1F
:1002300007E1192A05E1D880193218321732202A2D
:10024000080E202617C016F018C017F019C018F0B5
:1002500011D018520FE1080E205E175007E1080E6A
:10026000205E165002E1195010D0166A186E16C0A2
:1002700017F0166A18BE06D0D890163617361836FC
:100280002006F8D721AE189E205016C019F0166E21
:10029000185017C018F0176E1200F86A400E1F6E43
:1002A000AB6AAC6A7B6A7A6A7E6A7F6AC26AA66A4D
:1002B000A68E900EF26E010E926E936881903C0EA7
:1002C000C26EC16A8A0EC06E010E7E6E7F6AC280E7
:1002D000C282C2B2FED71ED0F2A203D0F292F28E38
:1002E00000D09292899292948984800E006E080EBA
:1002F000036EA00E016E0F0E026EC40E086E090E84
:10030000096EB80E116E0B0E126EB0DE92948994C7
:10031000819075D09292898292948984010E076EA1
:10032000F40E01DF9292899292948994000EE5DE98
:10033000266E12C027F026C016F027C017F061DF26
:10034000090E1D6E240E1C6E100E1B6E770E1A6E9B
:1003500008DF19C025F018C024F017C023F016C01C
:1003600022F0010E076E900EDEDE23BE09D0000ED5
:10037000255C000E2458200E2358800E225826E2B9
:1003800092948984010E076EF40ECDDE92948994C6
:10039000010E076EF40EC7DE92948984010E076E7B
:1003A000F40EC1DE92948994010E076EF40EBBDE4A
:1003B00092948984010E076EF40EB5DE92948994AE
:1003C000010E076EF40EAFDE1AD019D09292898218
:1003D000010E076EF40EA7DE92928992010E076E4F
:1003E000F40EA1DE92928982010E076EF40E9BDE5E
:1003F00092928992010E076EF40E95DE00D09292D1
:060400008982FDD7FFD741
:020000040030CA
:0300010006190ECF
:020005008180F8
:060008000FC00FE00F40E5
:00000001FF
